:020000040800F2
:10000000B8090020D5000008651E00087519000811
:1000100000000000000000000000000000000000E0
:10002000000000000000000000000000A321000804
:100030000000000000000000AD1E0008A52100081F
:10004000E7000008E7000008E7000008E7000008F4
:10005000E700000889010008E7000008E700000841
:10006000E7000008E7000008E7000008E7000008D4
:10007000E7000008E7000008E7000008E7000008C4
:10008000E7000008E7000008E7000008E7000008B4
:10009000E7000008E7000008E7000008E7000008A4
:1000A000E7000008B11E0008E7000008E7000008AC
:1000B000E7000008A5270008E7000008E70000089F
:1000C0000348854600F04EF8004800473D2F0008E1
:1000D000B80900200448804704480047FEE7FEE7CF
:1000E000FEE7FEE7FEE7FEE71D220008C10000086C
:1000F00030B50B46014600202022012409E00D46C0
:10010000D5409D4205D31D469540491B2546954047
:1001100040191546521E002DF1DC30BD03460B433D
:100120009B0703D009E008C9121F08C0042AFAD2AD
:1001300003E00B780370401C491C521EF9D2704733
:10014000D2B201E00270401C491EFBD2704700226F
:10015000F6E710B513460A4604461946FFF7F0FFC6
:10016000204610BD064C0125064E05E0E36807CC8D
:100170002B430C3C98471034B442F7D3FFF7A4FF4D
:100180008C460008AC46000810B5022000F042F88A
:1001900010BD70B50024014620314A78022A03D0F0
:1001A00004218163012416E0026813680E25AB4325
:1001B0001360026813685B085B0013600122056C22
:1001C0001346AB40C56B6B604A7000220A70416BEE
:1001D000002900D08847204670BD31B500F0E2F814
:1001E000009C0546601C00D0641C00F0DBF8401B3E
:1001F000A042FAD338BD000000B5022807D105207F
:1002000002F08CFD002802D001490120087200BDD7
:100210004800002010B504494A69024202D04861F2
:10022000FFF7EAFF10BD000000040140F8B500230D
:1002300093E0224601249C40A44622407ED04C6894
:10024000022C01D0122C0CD1DC08A40027183C6A27
:100250005D07ED0E0F26AE40B4430E69AE40264357
:100260003E6205685E000324B4400F79A543BF07D2
:10027000BF0FB7402F4307604D68012D05D0022DF9
:1002800003D0112D01D0122D0ED18568CF68A54362
:10029000B7402F43876047686546AF430D79ED0649
:1002A000ED0F9D403D434560C568A5438C68B44053
:1002B0002C43C4604C68E4004ED52B4CA569012644
:1002C0003543A561A4699D0834400094274CAD00D6
:1002D0002F19BC689D072E0F0F25B540AC4309258B
:1002E000ED06A84201D1002514E0214DA84201D11C
:1002F00001250FE01F4DA84201D102250AE01E4D45
:10030000A84201D1032505E01C4DA84201D10425D6
:1003100000E00525B5402543BD60194C25684E68B1
:100320009543F60300D51543256065684E689543EF
:10033000B60300D515436560A56800E00CE04E6883
:100340009543F60200D51543A560E5684E689543D0
:10035000B60200D51543E5605B1C0A681446DA4016
:1003600000D066E7F8BD0000001002400000014028
:100370000004004800080048000C00480010004835
:10038000000401400069084000D001207047426924
:100390004A4042617047002A01D081617047816202
:1003A0007047000001480068704700007C00002092
:1003B00070B5024640325378202B1CD11378012BA4
:1003C00019D00123137024245470046825689D43B8
:1003D0002560046825681E03B54325600468256808
:1003E0000D432560006801681943016020205070AA
:1003F0000020107070BD022070BD70B50246403202
:100400005378202B1BD11378012B18D001241470A2
:100410002423537003681D68A5431D6005682B687D
:100420000F263602B34309021943296000680168A8
:1004300021430160202050700020107070BD022008
:1004400070BD000070B5040006D0254640356878C0
:100450000026002802D005E0012070BD2E70204645
:1004600000F082F92420687020680168490849007A
:1004700001600F21606809068843216808612168CE
:100480008A680120C00382438A60E1680129A1686B
:1004900008D021229202114322689160E16802296A
:1004A00002D005E00143F7E701212268C90251604B
:1004B00021684A680F4B1A434A602168CA68824320
:1004C000CA60616920690843A1690902084321687B
:1004D000C860216AE06908432168086020680168F3
:1004E0000122114301606664202068702663AE70AB
:1004F000002070BD00800002FFB50446002083B0DC
:100500002546403501906A78202A7FD12268926979
:10051000D24312047AD52A78012A77D001222A7090
:1005200024226A7060648F05BF0DE06801280BD03B
:100530000520C002012138188902884321684860DB
:10054000FFF730FF064612E03148F3E70698401CFB
:100550000DD00698002805D0FFF724FF811B0698D0
:10056000814204D9202068700020287043E0206870
:100570008169C943890606D58069C043C00602D592
:100580006878A028E2D120688069069BC043C00635
:1005900000960ED500222021204601F07FFA002887
:1005A00029D121682020C86168700020287007B018
:1005B000F0BD00222021204601F070FA00281AD157
:1005C00020681021C16120682021C1610198411C6F
:1005D00001910599884214D1206841680122920353
:1005E000114341600096002220212046069B01F025
:1005F00055FA002802D00320D9E707E0216820201F
:10060000C8610199059881428FD3ABE70220CEE7FC
:1006100000200002FFB5054604464035687883B0E7
:10062000202876D10C98002874D00D98002871D01D
:10063000287801286DD001202870FFF7B3FE074607
:10064000012200901923D103204601F027FA002847
:1006500053D1212068704020A870002666640C9851
:1006600060620D98608566630E980090019704A9FA
:100670000EC9204601F0CAF9002804D0606C2E7023
:1006800004286AD039E0608DFF2805D9FF22228531
:1006900001231B06009606E0608D20850096208DC4
:1006A0000123C2B25B062046049901F0E5F93A46FF
:1006B00020460E9901F03DFA002803D0606C042812
:1006C0004BD01AE0606A411C616221680078886240
:1006D000608D401E6085208D401E0004000C20852A
:1006E00024D1608D002821D000970022802120464F
:1006F0000E9B01F0D3F9002802D0032007B0F0BD13
:10070000608DFF2807D9FF22228501231B06009652
:1007100008E024E021E0608D20850096208D0123F3
:10072000C2B25B062046049901F0A6F9608D00284C
:10073000BDD13A4620460E9901F0D4F90028BDD12A
:1007400020682021C16120684268064B1A4042603F
:100750006970AE702E700020D0E70120CEE7022035
:10076000CCE7000000E800FE00B500680E4987B045
:10077000884217D1032040030090122001900020EE
:100780000290032003900520049069460748FFF774
:100790004DFD0748C269012189050A43C261C0694C
:1007A0000840059007B000BD005800400004004814
:1007B0000010024070B504000FD021681348086093
:1007C00021681348086003CC41602068083C216818
:1007D0008860FFF7E7FD054608E0012070BDFFF7E0
:1007E000E1FD401B272801D9032070BD2068C068A7
:1007F0000028F4D120680269E1688A4201D00161D1
:1008000001E004490160002070BD0000CCCC000074
:1008100055550000AAAA00000068024901600020A6
:1008200070470000AAAA000002480168491C016044
:10083000704700007C00002010B5064801681022B7
:1008400011430160002000F007F800F017F80020C5
:1008500010BD00000020024010B5044600F078F9F9
:100860007D21C900FFF744FC00F0E2FD0022214693
:10087000501E00F02FF8002010BD000008B50F48F2
:100880008169012211438161816911400091C2692E
:1008900001040A43C261C069002208400090114669
:1008A000501F00F017F800221146901E00F012F8B9
:1008B00000221146501E00F00DF808BD0010024045
:1008C000C106C90E01208840014908607047000038
:1008D00000E100E010B501F0C7FA10BDF8B504461C
:1008E0000068434DC00352D5E8690026C00007D414
:1008F000E96928040143E961E969014001260091A1
:100900003C480168C90510D4016882151143016093
:10091000FFF748FD074604E0FFF744FDC01B6428CD
:1009200024D834480068C005F6D5286A03273F025A
:10093000384020D06168394081421CD0286A2A6A38
:10094000B843012109040A432A622A6A8A432A62B7
:100950002862C0070FD0FFF725FD009008E0FFF7E1
:1009600021FD0099411A2448814201D90320F8BD94
:10097000286A8007F3D5286A6168B843084328626B
:10098000002E04D0E869012109078843E861207836
:10099000C00705D0286BA168800880000843286341
:1009A0002078800706D5286B032109048843E16875
:1009B000084328632078800605D5286B10218843DA
:1009C0002169084328632068800305D5286B8021AE
:1009D0008843A169084328632088400505D5286B12
:1009E000402188436169084328630020F8BD000066
:1009F000001002400070004088130000F8B5054662
:100A00004E480E460068C007C00FB0420AD24B489D
:100A1000016849084900314301600068C007C00F00
:100A2000B04270D12878464C800705D56068F02127
:100A30008843A968084360602878C00753D0686875
:100A4000012817D0022818D0032819D02168890757
:100A5000002958DA61688908890001436160FFF75D
:100A6000A1FC69680746012913D002291DD003297A
:100A700027D034E021688903EAE721688901E7E7A4
:100A8000616BC903E4E7FFF78DFCC11B2D48814270
:100A900023D860680007800F0128F4D123E0FFF716
:100AA00081FCC11B2748814217D860680007800F6E
:100AB0000228F4D117E0FFF775FCC11B21488142E1
:100AC0000BD860680007800F0328F4D10BE0FFF714
:100AD00069FCC11B1B48814201D90320F8BD606835
:100AE0000007800FF3D115480168C907C90FB1424B
:100AF0000BD9016849084900314301600068C0070B
:100B0000C00FB04201D00120F8BD2878400706D5BB
:100B10006068072109028843E9680843606000F0C3
:100B20002DF86168084A0906090F515CC840074959
:100B300008600020FFF790FE0020F8BD0020024072
:100B40000010024088130000714600088000002059
:100B500001480068704700008000002004480549F3
:100B600000684968044A4905490F515CC84070470C
:100B700080000020001002408146000830B516A316
:100B80000FCB89B06C460FC417A30FCB0FC41A4903
:100B90004A680C20144604401848042C05D0184B11
:100BA000082C04D00C2C00D1184609B030BD94029A
:100BB000240F6D462C5DC96A04AD0907090FD203E5
:100BC000695C920F022A02D0032A00D11846FFF76F
:100BD0008FFA6043E9E700000203040506070809ED
:100BE0000A0B0C0D0E0F1010010203040506070876
:100BF000090A0B0C0D0E0F100010024000127A00B3
:100C0000006CDC02FEB504460078F04EF04DC007E3
:100C100048D068680007800F01281FD06868000767
:100C2000800F022804D16868C003800F022815D005
:100C30006168012919D001208004002901D005290B
:100C400017D02968B1432960296881432960606809
:100C500000281BD0FFF7A6FB074613E02868800397
:100C600020D56068002876D01CE0286830432860D2
:100C7000EDE7296801432960F7E7FFF793FBC01B05
:100C8000642869D828688003F7D50BE0FFF78AFB52
:100C9000074604E0FFF786FBC01B6428F1D82868EC
:100CA0008003F7D4207880073ED568680007800F5E
:100CB00014D068680007800F022804D16868C00358
:100CC000800F01280AD0E068002828681DD0012183
:100CD00008432860FFF766FB07460BE0286880079B
:100CE0000BD5E068012836D107E0FFF75BFBC01B9E
:100CF0000228C6D828688007F7D52868F8218843D5
:100D00002169C900084328600EE0400840002860BF
:100D1000FFF748FB074604E0FFF744FBC01B02282F
:100D2000AFD828688007F7D42078000724D5E06979
:100D30000028686A11D0012108436862FFF732FB7E
:100D4000074604E0FFF72EFBC01B022899D8686A0B
:100D50008007F7D510E036E1D1E040084000686236
:100D6000FFF720FB074604E0FFF71CFBC01B02282F
:100D700087D8686A8007F7D42078042740070028BE
:100D800061DA00200190E869C00008D4E969B8067A
:100D90000143E961E96901400120009101908D481A
:100DA0000168C90511D40168821511430160FFF77C
:100DB000F9FA009005E0FFF7F5FA0099401A642867
:100DC00097D884480068C005F5D5A06801280AD0E6
:100DD000002801D0052811D0286A40084000286268
:100DE000286AB84302E0286A012108432862A06803
:100DF000002812D0FFF7D6FA00900AE0286A38439C
:100E00002862F0E7FFF7CEFA0099411A7248814252
:100E100075D8286A8007F5D50DE0FFF7C3FA009072
:100E200006E0FFF7BFFA0099411A6B48814266D885
:100E3000286A8007F5D40198002804D0E9690120C8
:100E400000078143E9612078C00635D56069012833
:100E50000CD0401D686B24D038436863686B400831
:100E600040006863FFF79EFA074622E0686B38434C
:100E70006863686B012108436863FFF793FA0746CC
:100E800004E0FFF78FFAC01B022838D8686B800790
:100E9000F7D5686BF8218843A169C90008436863E6
:100EA0000AE0B8436863F4E7FFF77CFAC01B022846
:100EB00025D8686B8007F7D42078800637D5686816
:100EC0000007800F032813D068680007800F0228EE
:100ED00004D16868C003800F032809D0206A002865
:100EE000686B16D030436863FFF75CFA06460CE087
:100EF000686BC0031BD5206A012864D117E05BE052
:100F0000FFF750FA801B022856D8686BC003F7D54C
:100F10000DE0B0436863FFF745FA064604E0FFF7CB
:100F200041FA801B022847D8686BC003F7D4606A77
:100F3000002846D069680907890F022943D0012695
:100F400036060228286805D0B0432860FFF72AFA41
:100F5000044633E0B0432860FFF724FA074604E074
:100F6000FFF720FAC01B022826D828688001F7D492
:100F7000E86A216B000900010843E862A16AE06A9F
:100F8000084369687B22D20391430843686028685C
:100F900030432860FFF706FA044604E0FFF702FA40
:100FA000001B022808D828688001F7D509E0FFF760
:100FB000F9F9001B022801D90320FEBD2868800131
:100FC000F5D40020FEBD0120FEBD000000000100A0
:100FD00000100240007000408813000070470000BD
:100FE000F8B504460068426881684B0605D4CB0713
:100FF00003D0530601D5E16C04E08B0705D5130639
:1010000003D5216D20468847F8BDFF23613319427F
:10101000FAD09306F8D523464D064033002D09DA61
:101020005D7F032D3CD0256E042635432566C568BB
:10103000856800958E060125002E08DA266E2E435F
:1010400026668668009606684027BE430660C80587
:1010500006D5206E0821084320662068806800902D
:10106000206E0028D0D020684168E026B14341605E
:101070005D77900718D02068416889088900416031
:10108000A06D0B4D002803D04563A06DFFF781F8DC
:10109000606D0028B8D04563606DFFF77AF8F8BD41
:1010A000C16880680090F8BD2046FFF797FFF8BD43
:1010B00023200008F8B5040007D000262546403557
:1010C000A662687F002802D005E00120F8BD2E77D7
:1010D000204600F04BF802236B772068016840221D
:1010E000914301600721E0680902884201D900228A
:1010F00001E0012212030F273F02B84202D08842CA
:1011000000D0A662276B002F05D1884201D9236346
:1011100001E001202063A1686068636908432169D8
:10112000194308430123A1695B0219400843E1699F
:101130000843216A0843A16A084321680860616B7B
:10114000606AA36908431B0C0427E1683B4019430C
:1011500008432168104348602068C1697A029143BE
:10116000C1612666012068770020F8BD00B50068DF
:10117000114987B088421DD11048826981140A4301
:101180008261806908400590F02000900220019063
:101190000021032003900291049109206946C006B2
:1011A000FFF744F8002211461920FFF793FB19209E
:1011B000FFF786FB07B000BD003001400010024081
:1011C00070470000F0B504468C464034217F00256E
:1011D000C768964601290CD001212177667F4168B6
:1011E000012E0CD0CA1FFD3A07D18168002904D115
:1011F00001E00220F0BD042E01D0022540E061464E
:1012000000291BD07146002918D0002B16D0617F11
:10121000042901D0052161770021016661468163BF
:101220008387C38771460164A380E3800721090295
:101230008F4205D9144AC264144A04E001251FE014
:10124000134AC264134A0265012212038F4202D874
:10125000E188022903D301684B68934302E00168E7
:101260004B6813434B6001684A68E0231A434A60A5
:1012700000680168490603D40168402211430160F7
:10128000002020772846F0BDC11E0008551F000829
:10129000F71E0008891F0008F8B501220920D103B4
:1012A000C006FFF778F856492022881AFEF736FF65
:1012B000534C0127203C2078524EDE2801D0777213
:1012C00091E0A07808280BD0092810D000250B2821
:1012D00030D003284AD001284FD002287AD082E0AB
:1012E0004748A2792179203001F022FD7BE0617925
:1012F000207901F071FB424A2C321060E179A0792B
:1013000001F06AFB40425060207A3D494042107231
:10131000607A5072607B9072A07B1073E07BD07219
:10132000207C5073607C907336482C31243001F05F
:10133000FFFF58E0324821794C30017061794170EB
:10134000A1798170E179C170057145718571C571AF
:10135000217A0172617A4172A17A8172E17AC17255
:10136000014628482C3001F065FB3CE001210022B9
:1013700049032548FFF70FF835E021482021403880
:10138000FEF7E5FE1E48CD214038017061784170BE
:1013900080238370C7703178017145710521817197
:1013A0000721C171082200210546A1356C5C002C83
:1013B0000CD0022C02D0012C03D005E0815403E0B4
:1013C00008E00C461C438454521CD2B2491C10291C
:1013D000ECDB08E00325605D002804D001F026FC6A
:1013E0006D1C202DF7DB064A2023114640390748A3
:1013F000FFF7E8FE01F032FF054940187061F8BDC3
:101400004003002048000020000800487C01002024
:1014100010270000042204490428086902D09043E0
:10142000086170471043FBE700E000E070470000F0
:10143000094910B5401E884201D9012010BD074C52
:1014400060610321081F00F00FFD0020A06107204C
:101450002061002010BD0000FFFFFF0000E000E061
:1014600010B5FFF7E3FF10BD70B502462032137FC1
:10147000012B1BD00123137702245477046865687D
:101480007026B5436560046865680E68354365601D
:101490000468A5688026B543A5600068846849682B
:1014A0000C43846053770020107770BD022070BD1C
:1014B00070B5040005D025462035687F002802D08D
:1014C00006E0012070BD00202877204600F00AF8D1
:1014D00002206877211D206800F0CEFE0120687789
:1014E000002070BD08B5006801218907884207D136
:1014F0000448C16901221143C161C06910400090D4
:1015000008BD0000001002400222014620314A7747
:101510000268136801200343136048770020704776
:10152000F8B5054604462035287F012817D0012745
:101530002F7702206877226890687726FF23B043D0
:101540001B02984390600868502837D00EDC202892
:1015500057D006DC00284ED0102840D14EE00220A3
:10156000F8BD302850D0402839D13CE060282DD03B
:10157000702817D001221203801A0ED090422ED16B
:10158000CB684A688968206800F0C0FE20688168DE
:10159000012292031143816021E020688168C9081B
:1015A000C900F8E7CB684A688968206800F0AEFE99
:1015B00021688868B0433043886010E0CA68496891
:1015C000206800F0B6FE5021206806E0CA6849682D
:1015D000206800F0BFFE6021206800F0A2FE6F7757
:1015E00000202877F8BDCA684968206800F0A1FE8D
:1015F00040212068F1E700212068EEE710212068F3
:10160000EBE720212068E8E730212068E5E7704714
:1016100070470000F8B503680446D86919680507E3
:101620002D0F07D1820605D58A0603D5204600F086
:1016300069FFF8BD9A68002D64D0D507ED0FFF262D
:1016400021360E402E435DD0C60706D0CE0504D508
:1016500001261E62E36E3343E366870702230426F6
:10166000002F06DAD70704D027683B62E76E3743BE
:10167000E766470706D5D20704D022681662E26EF5
:101680001A43E266020709D520220A402A4305D000
:10169000236808221A62E36E1343E366E26E002AAF
:1016A000C7D0800604D5880602D5204600F02AFF60
:1016B000E06E000703D42068806840061CD52046F1
:1016C00000F004FF20688168490611D58168402236
:1016D00091438160606E00280AD01A494163606EB0
:1016E000FEF757FD0028A4D0606E416B8847F8BD17
:1016F0002046FFF78DFFF8BD2046FFF789FF002049
:10170000E066F8BDC5020DD552020BD501200005DB
:101710001862202120466030417281722046FFF716
:1017200076FFF8BD020605D50A0603D5204600F06F
:10173000D5FFF8BD4006FCD54806FAD5204600F096
:10174000D4FEF8BDB924000870B5040005D02546C4
:101750006035687A002802D006E0012070BD0020C4
:101760002872204600F026F824206872206801685C
:10177000490849000160204600F002FF0128EDD031
:10178000606A002802D0204600F0F7FD206841681A
:101790000922D20291434160206881682A22914344
:1017A000816020680168012211430160204600F039
:1017B00049FE70BD30B51F4D046800211E4802224D
:1017C000032387B0AC4214D1856954032543856156
:1017D00080690291204005905802009001200490F9
:1017E0000920039301926946C006FEF71FFD07B06A
:1017F00030BD124DAC42FAD1C5690124A404254381
:10180000C561C069029120400590032080020090CC
:10181000042004900393019269460948FEF706FDEF
:10182000002201211D20FFF755F81D20FFF748F881
:10183000DDE7000000380140001002400048004091
:10184000000400487047FFB5064604466036707ACB
:1018500083B00D46202858D1002D0CD005980028C3
:1018600009D00120A1680003814207D12069002826
:1018700004D1E80702D0012007B0F0BD307A01287A
:1018800043D0012030720020E06621207072FEF704
:1018900089FD01902746403705983882059878825F
:1018A00018E0788A401E78820698009000228021F5
:1018B0002046019B00F045FF002818D10120A168B7
:1018C0000003814202D12069002812D021682878C3
:1018D00008856D1C788A0028E3D1069800900022C4
:1018E00040212046019B00F02CFF002808D0032057
:1018F000C2E728882168C005C00D0885AD1CE9E74E
:101900002020707200203072B6E70220B4E730B5B4
:10191000034660335C7A202C23D100290BD0002AA7
:1019200009D0012584682D03AC4206D10469002C3E
:1019300003D1CC0701D0012030BD1C7A012C10D07E
:10194000C164014640310A824A820021C1662122D7
:101950005A721972006801688022114301600020E8
:1019600030BD022030BD0000014900208872704760
:1019700048000020FEE701688A69D243920701D43B
:1019800000228A6200688169C943C90703D081695E
:101990000122114381617047F7B5044600680E4685
:1019A0008069C043C0062CD42027254640352068D6
:1019B0008069C04380060FD5701CF8D0002E05D07A
:1019C000FEF7F0FC0299401AB042F0D96F70002087
:1019D000A87028700320FEBD21681020C86120680F
:1019E000C7612046FFF7C7FF20684168064A1140DB
:1019F0004160042060646F700020A870287001208E
:101A0000FEBD0020FEBD000000E800FEF8B5044663
:101A10000120164640031D46DAB2C3020090079F1C
:101A2000204600F029F83A462046069900F081F851
:101A3000002803D0606C04281BD018E02846F5B2BB
:101A4000012809D02168300A88623A462046069962
:101A500000F06FF80028EDD1206885620097002221
:101A600080212046069B00F019F8002800D00320B2
:101A7000F8BD0120F8BD000070B50568049C6868D9
:101A80008905890D1204044E114319433040214346
:101A90000143696070BD0000009800FCF8B51C4669
:101AA00017460E46054611E0601C0FD0002C05D0ED
:101AB000FEF778FC0699401AA04207D9202040354D
:101AC00068700020A87028700320F8BD286881691C
:101AD0003046884304D00020B842E5D00020F8BD4D
:101AE0000120F9E770B516460D4604461AE0324665
:101AF00029462046FFF750FF002801D0012070BD85
:101B0000002D04D0FEF74EFC801BA8420AD9616C60
:101B1000202001436164403460700020A070207078
:101B2000032070BD20688069C0438006DFD4002098
:101B300070BD70B516460D4604461CE03246294677
:101B40002046FFF729FF002801D0012070BD681C46
:101B500011D0002D04D0FEF725FC801BA8420AD925
:101B6000616C202001436164403460700020A070EB
:101B70002070032070BD20688069C0438007DDD4D9
:101B8000002070BDF0B5504887B041690120C00405
:101B90004D4A014351615169014005915169C000AD
:101BA000014351615169014005915169401101435F
:101BB000516151690140104605914169012080043D
:101BC00001435161516944110140059100222146B0
:101BD0003E48FEF7E0FB0326B603012231463B48B0
:101BE000FEF7D9FB012203213948FEF7D4FB394F18
:101BF000092000223946C006FEF7CDFBCD21012287
:101C000089003548FEF7C7FB002208213248FEF75D
:101C1000C2FB0094002401250195029469462B48DB
:101C20000394FEF703FB00961126029469462748A9
:101C300001960394FEF7FAFA032000900294694695
:101C4000019603942248FEF7F1FA092002946946AE
:101C5000C006009701950394FEF7E8FA1F48022793
:101C600001906946009702941B48FEF7DFFACD20E9
:101C70008000009002946946019603941648FEF78E
:101C8000D5FAE8036A4691C269461348FEF7CEFAD0
:101C900028026A4691C209206946C006FEF7C6FAC4
:101CA0000820009002946946019503940A48FEF7C3
:101CB000BDFA002202210520FEF70CFE0520FEF7EA
:101CC000FFFD07B0F0BD0000001002400008004812
:101CD00000140048018000000004004800002110AA
:101CE00010B512481049016011494160002181601E
:101CF0000161416181610122C161C2600162FEF73F
:101D0000A1FB002800D0FEE700210848FEF750FBA9
:101D1000002800D0FEE700210448FEF76EFB0028F3
:101D200000D0FEE710BD0000005800402001002058
:101D30005D3E302010B50D480B4901600021416027
:101D40008160016141618161072201621202416289
:101D5000C260816207220163C2624163FFF7AAF990
:101D6000002800D0FEE710BD003001407C010020BB
:101D700010B50121124886B08907016000242F2187
:101D8000846041600461611E8461C160FFF790FB63
:101D9000002800D0FEE701200003009069460848B3
:101DA000FFF7BEFB002800D0FEE7049404A9044816
:101DB0000594FFF759FB002800D0FEE706B010BDE0
:101DC000E001002010B50F480D490160E1214902F2
:101DD00041600D498989402901D00C4941600021A9
:101DE0008160C16001618161C1610C220162426157
:101DF00041620448FFF7A8FC002800D0FEE710BDB0
:101E00000038014020020020480000203EFA020075
:101E100010B51248104901604B2109014160104979
:101E20008989402902D07F21090141600021C160D8
:101E3000016181610C22C161426101623021416214
:101E40000121090381634900C1630448FFF77CFC59
:101E5000002800D0FEE710BD00480040900200209E
:101E600048000020704700008307FF22DB0E9A40E5
:101E70008907090E994000280BDA0007000F08387F
:101E8000830808489B001818C36993430B43C36138
:101E90007047830804489B001B1818689043084348
:101EA0001860704700ED00E000E400E070470000BB
:101EB00010B50248FFF794F810BD00007C01002027
:101EC00010B50168C968026C1180016C891C01643D
:101ED00001464031CA88521ECA80C988002909D1EA
:101EE00001684A6840239A434A60C18F002901D1A2
:101EF00000F06EF810BD10B501464031CC88036883
:101F0000026C012C11D9DB681380026C921C0264F4
:101F1000CA88921ECA80CA88012A0DD102685368F5
:101F2000012424032343536006E01C7B531C0364F9
:101F30001470CA88521ECA80C988002909D1016854
:101F40004A6860239A434A60C18F002901D100F09A
:101F50003FF810BD10B5816B02680988D160816BB4
:101F6000891C8163C18F491EC187C18F00290AD195
:101F700001684A6880239A434A604621095A002929
:101F800001D100F025F810BD10B5C38F0268816B38
:101F9000022B07D30988D160816B891C8163C18FB3
:101FA000891E05E04B1C836309781173C18F491E9C
:101FB000C187C18F00290AD101684A6880239A43EA
:101FC0004A604621095A002901D100F001F810BDEC
:101FD00070B50446FEF7E6F9024620684168202500
:101FE000A94341606421204600F024F8002802D073
:101FF000206E28432066226E204601214030002AB0
:1020000004D041772046FEF7E9FF70BD427F41775B
:10201000042A204602D0FFF73FF970BDFFF7D0F841
:1020200070BD10B5406A002146221152C187FEF7EB
:10203000D5FF10BDF8B50F460B461546009203219B
:1020400004460022C90200F01BF82026002812D105
:102050003B46002280212046009500F05CF80028D5
:1020600009D103213B46002249022046009500F099
:1020700007F8002803D0206E304320660320F8BD07
:10208000F8B51D4617460E4604463DE003214902B9
:102090008E4205D1002F03D1017B68460170007884
:1020A000681C31D0002D05D0FEF77CF90699401A46
:1020B000A84229D320684168E022914341606068CA
:1020C000C11FFD390CD10121A068C903884202D08B
:1020D0004911884204D1206801684022914301607F
:1020E0000120A16A4003814207D121680A68824326
:1020F0000A6021680A6802430A6001204034607760
:10210000002020770320F8BD206881683140B94263
:10211000BCD10020F8BDF8B51D4617460E46044652
:1021200033E0681C31D0002D05D0FEF73BF906994D
:10213000401AA84229D320684168E02291434160B7
:102140006068C11FFD390CD10121A068C903884214
:1021500002D04911884204D120680168402291438D
:1021600001600120A16A4003814207D121680A6809
:1021700082430A6021680A6802430A6001204034F1
:102180006077002020770320F8BD20688168304602
:10219000884304D00020B842C3D10020F8BD0120FC
:1021A000F9E7704710B5FEF73FFBFFF759F910BD8F
:1021B00030B599B028200125002400900895079596
:1021C00009946846FEF71EFD002800D0FEE70720B0
:1021D0000D9003200E900F94012110940DA8FEF78E
:1021E0000DFC002800D0FEE7119511A81395FEF70D
:1021F00075FB002800D0FEE7FEF7AAFC7D21C90090
:10220000FDF776FFFFF714F90420FFF703F900222A
:102210001146501EFEF75EFB19B030BD1248016832
:102220000122114301604168104A11404160016878
:102230000F4A11400160016801229204914301603C
:1022400041683F22120491434160C16A09090901B2
:10225000C162016B074A11400163416B49084900A3
:102260004163002181607047001002400CB8FF08F4
:10227000FFFFF6FE2CFEFCFFF0B502681D4B0124AB
:10228000A4071D4D984203D0A04201D0A84203D11B
:102290007026B2434E683243184E194F98420DD003
:1022A000A0420BD0A84209D0164CA04206D0B042A2
:1022B00004D0B84202D0144CA04204D1032424021A
:1022C000A243CC6822438024A2434C69224302608B
:1022D0008A68C2620A688262984206D0B04204D01C
:1022E000B84202D0084A904201D109690163012134
:1022F0004161F0BD002C014000040040004001405D
:1023000000440140002000400048014030B584688E
:10231000FF252D021B021343AC430B432343836071
:1023200030BD826870239A430A4307210A438260C2
:10233000704730B5036A046A640864000462846903
:10234000F025AC43120122430A24A3430B438261CC
:10235000036230BD30B5036A1024A343036284696D
:10236000036A0F252D031203AC432243A024A34389
:10237000090119438261016230BD10B5818CC90722
:1023800007D001684A6801235B049A43836A1A43B1
:102390004A60818C890707D501684A6801231B04BC
:1023A0009A43C36A1A434A60818C490707D501687A
:1023B0004A6801239B049A43036B1A434A60818C49
:1023C000090707D501684A680123DB039A43436B79
:1023D0001A434A60818CC90607D5026891680123B7
:1023E0001B039943836B19439160818C890607D540
:1023F00001688A6801235B039A43C36B1A438A60AE
:10240000818C490612D503685A6801210905046CBC
:102410008A4322435A60026C8A4207D1026851689B
:1024200003235B059943436C19435160818C090672
:1024300007D501684A680123DB04806C9A43024394
:102440004A6010BDF8B500260446C666FDF7AAFF2F
:10245000054616492068884202D0154988421DD198
:102460000068144F000709D501212B4600224905B9
:102470002046009700F065F900280DD1206800681B
:1024800040070BD501212B460022890520460097E5
:1024900000F057F9002801D00320F8BD2020603457
:1024A0006072A07226720020F8BD00000038014062
:1024B00000440040FFFFFF0110B5406A00220146C2
:1024C00040314A834A82FFF7A3F810BD01680A68C9
:1024D000FF2321339A430A6001688A685208520038
:1024E0008A60202160308172704710B501680A68E7
:1024F00040239A430A60202269210A54FFF734FAE4
:10250000002010BD70B50246403203466033948B04
:102510009D7A0168222D05D08869082210438861C0
:10252000022070BD898C012685683603B54202D130
:102530000569002D0BD02140446D651C4565217057
:10254000518B491E0904090C518307D015E0456DD4
:1025500021402980416D891C4165F1E701680A68C5
:10256000FF242134A2430A6001688A68520852009D
:102570008A6020219972FFF765F9002070BD000084
:10258000F8B504462369A268E5691A436369102017
:102590002B43002125681A432B680E46474F3B40CA
:1025A00013432B6023685A6803252D03AA43E5686B
:1025B0002A435A60236AA26925681A43AB680B272D
:1025C0003F02BB431343AB603D4F25683D4B0203C5
:1025D000BD420AD11B6B9B079B0F20D0012B14D04F
:1025E000022B14D0032B1BD10DE0374FBD4210D16D
:1025F0001B6B03273F043B4011D09B1A05D09B1A4D
:1026000005D093420CD102200AE0042008E0082003
:1026100006E02E4B9D4202D02D4B9D4200D1002062
:102620000123E769DB039F4222D100280CD0022856
:102630000DD0042813D0082817D001260A0912014A
:102640000807400F10432EE0FEF788FA09E06168A2
:10265000204A48088018FDF74BFD81B2EEE7FEF7EF
:102660008DFA616840004A08F4E761684808F1E7BC
:10267000002808D0022809D004280CD0082815D03A
:1026800001263046F8BDFEF769FA06E06168124A95
:10269000480880180DE0FEF771FA61684A08801852
:1026A000FDF726FD80B22168C860EAE76168480846
:1026B000C018FDF71DFD80B2E860E2E7F369FFEFA7
:1026C0000038014000100240004400400048004033
:1026D000004C00400024F40000127A006921095CDB
:1026E000212901D00220704702464032518A002938
:1026F00012D0012381681B03994202D1016900298C
:1027000015D0C16C4B1CC364006809780185508AE0
:10271000401E50820020704701680A6880239A4357
:102720000A6000680168402211430160F2E7C16C51
:1027300003680988C905C90D1985C16C891CC16464
:10274000E5E7FFB581B017460E4604460A9D1DE039
:10275000681C1BD0002D05D0FDF724FE0499401AFB
:10276000A84213D920680168FF22A1329143016079
:1027700020688168490849008160202060346072C7
:10278000A07200202072032005B0F0BD2068C1694E
:102790003046884304D00020B842D9D00020F3E767
:1027A0000120F9E710B50248FEF734FF10BD000024
:1027B000900200200FB410B503A9044B044A0298FC
:1027C00000F024F810BC08BC04B018471D2A00080B
:1027D0008400002030B47446641E2578641CAB422B
:1027E00000D21D46635D5B00E31830BC184702E071
:1027F00008C8121F08C1002AFAD17047704700208C
:1028000001E001C1121F002AFBD17047FFB58DB056
:102810000F460546002606E025280AD0109A0F9993
:1028200090476D1C761C28780028F5D1304611B0F1
:10283000F0BD00240121674A009400E004436D1CB0
:102840002B780846203B98401042F7D128782E2854
:1028500015D10420044368786D1C2A280AD101CFC1
:102860006D1C00900BE000990A225143303940184A
:102870006D1C00902878014630390929F3D9287851
:10288000692843D006DC0028D0D063280BD0642808
:1028900004D13BE073280FD075284CD0109A0F99C3
:1028A0009047761C94E03878694608720020487298
:1028B00002A80190012003E0386801900020C04385
:1028C0003F1D61070CD5002400E0641C00998C4278
:1028D0000FDA8442F9DB0199095D0029F5D108E09E
:1028E000002400E0641C8442FCDB0199095D00299E
:1028F000F8D1361907E0019801990078491C019137
:10290000109A0F999047641EF5D261E00A20019059
:1029100001CF002802DA40422D2102E0210504D532
:102920002B216A461172012103E0E10701D0202129
:10293000F7E70C9104E00A20019001CF00210C91EF
:102940000BA90B9108E00199FDF7D2FB0A460B9900
:102950003032491E0B910A700028F4D10B9803A95C
:10296000081A20300190600701D5009801E001208D
:1029700000900199884203DD01460198081A00E0A1
:1029800000200024009006E002A8109A005D0F9934
:102990009047641C761C0C988442F5DB04E0109A86
:1029A00030200F999047761C0099481E009000290E
:1029B000F5DC08E00B980B990078491C0B91109AF4
:1029C0000F999047761C0199481E01900029F1DC6F
:1029D0006D1C28E7092801000902014308B270476D
:1029E00002687F2A01DD7F2103E07E21C9438A42FC
:1029F00000DA0160704700B5014600F02FFC411875
:102A000000F02CFC8842FBD300BD000010B5024949
:102A10000860FEF779FD10BD0000002013B56423A7
:102A2000012269460248FEF70EFF00981CBD000017
:102A30002002002010B50B46044600F01DF80028C7
:102A400001D0012010BD20780C2261685043081885
:102A50001946FDF763FB2078401C4007400F2070AB
:102A6000002010BD10B50446602000F07DFB6060C2
:102A7000204600F020F810BD41780078401C400747
:102A8000400F814201D101207047002070474178FA
:102A90000278914201D10020704740680C225143D6
:102AA0004018704741780278914203D0491C490789
:102AB000490F4170704710B50021017041704068A6
:102AC0006021FDF744FB10BD70B52548FFF7DFFF1F
:102AD00004003BD02078002839D00022214E02216A
:102AE0003046FDF758FC6078002832D000221E4D99
:102AF0000121C9032846FDF74EFCA07800282AD002
:102B0000002201213046FDF746FCE078002824D061
:102B10000022012189032846FDF73DFC207AFF258C
:102B2000291A032000F07EFB607A291A002000F0A9
:102B300079FBA07A291A022000F074FBE07A291AA6
:102B4000012000F06FFB0648FFF7ACFF70BD0122CB
:102B5000C4E70122CBE70122D3E70122D9E7000035
:102B600074000020001400480008004870B50C4CA8
:102B7000012202212046FDF70EFC0A4D0122D1035D
:102B80002846FDF708FC012211462046FDF703FC0C
:102B9000012291032846FDF7FEFB00F02BFB70BDE0
:102BA000001400480008004870B505460020086081
:102BB00048600872487288720873C87248730C467D
:102BC0008873284600F0E0FB002827D021680268BF
:102BD000891821606168426889186160217A027AE7
:102BE00089182172617A427A89186172A17A827A8F
:102BF0001143A172217B027B11432173E17AC27AD6
:102C00001143E172617B427B11436173A17B807B45
:102C10000143A173284600F0C1FBD2E72046FFF72D
:102C2000DFFE201DFFF7DCFE70BD000070B544061E
:102C3000C109640EC901102C2BD2254D285D002836
:102C400027D0002926D0022823D122482300FFF7CD
:102C5000C1FD091E060D1E10161E1C191E00FF23A5
:102C600001330246590000F039FC10E001F010FB7E
:102C70000DE010230246202101F09EF807E000F04D
:102C8000A1FB04E000F0AAFB01E0FFF76FFF0120C9
:102C9000285570BD0128FCD1022028552300FFF7DC
:102CA00099FD0805060B050E05051305F1E700F073
:102CB000D9FD00F0E7FD70BD01F03AFB70BD01F0F9
:102CC00015F901F003F970BDFFF750FF70BD00006A
:102CD000A103002000040048002802D0ED2901D300
:102CE000002070470B4882780B48012A04D0022A42
:102CF00006D0032A08D00BE08E2909D2042206E070
:102D00008E2905D2022202E08E2901D203224254EA
:102D1000012070470400002090000020102803D2FA
:102D20000249085C012800D000207047A103002060
:102D300010B50C46034600F01FF8002801D0012012
:102D400010BD197858684454197898684254187816
:102D5000401C4007400F1870002010BD10B50446FD
:102D6000082000F001FA6060082000F0FDF9A06082
:102D7000204600F025F810BD41780078401C40073F
:102D8000400F814201D1012070470020704710B5EB
:102D900043780478A34201D1012010BD4468E35C6C
:102DA0000B7081684078085C1070002010BD41787D
:102DB0000278914203D0491C4907490F417070477E
:102DC00010B5044600202070607008216068FDF78F
:102DD000BEF90821A068FDF7BAF910BDF3B581B0BE
:102DE0000746FF2069460870524C3946A078FFF725
:102DF00073FF002814D10026ED3FA67001250321A2
:102E000002224D483B00FFF7E5FC1388820B660B5E
:102E1000585049403D36302A2422201E0B0F0B000B
:102E200014220121FA2075E014220121FA2000F079
:102E3000A5FD00F027FDFF204E30FDF7CEF9FA2268
:102E40000021AA2066E0A170EAE7A270E8E7A57079
:102E5000E6E700214554491C8E29FBDBE0E7002210
:102E60008154521C8E2AFBDBDAE700214254491CB4
:102E70008E29FBDBD4E7002104224254491C8E2911
:102E8000FBDBCDE700F0FEFCCAE700F0FBFC142200
:102E90000121FA2000F072FD6670FEBD14220121AE
:102EA000FA2000F06BFD6570FEBD14220121FA20AE
:102EB00000F064FD1E21684636E014220121FA204C
:102EC00000F05CFD14220021AB2000F057FD14221D
:102ED000002183201EE014220121FA2000F04EFD83
:102EE0001E21684600F040FC0028DDD1142201219B
:102EF000FA2000F043FD68460078002803D003283C
:102F0000D2D82070FEBD14220021207802E01422C5
:102F10000121EE2000F032FDFEBD14220121FA2035
:102F200000F02CFD1E21029800F01EFC00288BD022
:102F3000FEBD000004000020900000201CB5714878
:102F4000714C8089A081FDF777FCFFF731F9FEF71E
:102F500019FEFEF7C5FEFEF7EDFEFEF709FFFEF7D0
:102F600031FFFEF755FF6A4868490160032141605F
:102F70006849C1608160FDF71DFC002800D0FEE7B4
:102F80006348FDF749FC07210520019100900023CB
:102F90002278614961A0FFF70DFC5D487430FFF7AE
:102FA00035FD00F067FAFF260136614D77002A46AD
:102FB00033463946104600F091FA2A4633463946E0
:102FC000104601F06FF92A4610232021104600F028
:102FD000F3FE0220FFF7A2FE002801D001F058F90D
:102FE0005448FFF7BBFE4848243000F0B7F9464884
:102FF0002C30FFF737FD00F0FDF84E4820216038F7
:10300000FDF7A5F84B4A4248203A114620234039A3
:103010001030FEF7D7F8A18947A0FFF7CBFB00F0EF
:10302000D9F8002812D148A0FFF7C4FB00270821D7
:103030002846FDF7ACF93220FDF7CFF87F1C0A2FA8
:10304000F5DB012208212846FDF7A5F90927FF062F
:103050002F48FDF7E1FB00F001F96169884205D9CD
:1030600001210022C9033846FDF795F90420FFF736
:1030700055FE002809D00121C9032846FDF782F931
:10308000002802D000F05EFF0EE00520FFF746FEAC
:10309000002802D000F0EAF806E00820FFF73EFE24
:1030A000002801D000F0A4F90120FFF737FE002826
:1030B0000FD031463846FDF765F9002809D000F0F9
:1030C000F3FB002812D0002201213846FDF763F9F6
:1030D0000CE00220FFF722FE002807D031463846D8
:1030E000FDF750F9002801D001F042F90720FFF761
:1030F00015FE002801D0FFF7E7FC607A0028A7D072
:1031000001F052F8C0F7FF1F4800002000300040D7
:103110006C010020FF0F00003A46000825730A7278
:1031200065762564207625642E25642E25640A00A4
:103130000004004860030020666C6173685F736977
:103140007A653A2025640A004469676974616C20D5
:10315000706F74206E6F7420726573706F6E646927
:103160006E67210A00000000F0B50B30C108C900ED
:10317000144F0026144A0FE003688B420BD38B4296
:1031800005D95C1A4318456830C3083B00E0436822
:10319000136002C004E0021D10680028ECD1304624
:1031A000002803D13868002801D00020F0BD064A6D
:1031B00006481060064A121AD208D20044C0012004
:1031C0003860D7E78C00002088000020BC03002076
:1031D000B805002010B56423012258210448FDF7EA
:1031E0008BF9002801D0002010BD012010BD000087
:1031F0002001002070B50A4C002204212046FDF772
:10320000CAF87D25ED002846FFF7F5FB01220421D1
:103210002046FDF7C0F82846FFF7EDFB70BD000023
:103220000004004803B583B0042802D3FF2005B092
:1032300000BD08496423085C01210007020E04A8B0
:103240000293019100900B4658210348FDF7E2F9E3
:10325000EDE7000036460008200100200248006823
:103260000068406A704700000000002070B52E4CD6
:10327000207A00260125002808D04D20E071012287
:10328000E11D2A48FEF743FBA5722672264824302A
:1032900000F07AF8002845D0A07A002842D12349CE
:1032A0002148EC312430FFF77FFC1F48C0210E304D
:1032B0000680867001701D49EC318A7A002A01D09F
:1032C000E02202700A7B002A03D0027810231A43FE
:1032D00002700A88898812B2494209B20B0603D5E6
:1032E00003780826334303704B0603D5037804267E
:1032F00033430370130603D5037802263343037068
:10330000530602D503782B4303709206920E427047
:103310008906890E8170044903220E310348FEF7A5
:10332000F6FAA57270BD000048000020900200204F
:1033300030B50B46024600F01CF8002801D00120F1
:1033400030BD11785068090140183ACB3AC0107866
:10335000401C0007000F1070002030BD10B504465F
:10336000FF200130FFF700FF6060204600F01FF8EB
:1033700010BD41780078401C0007000F814201D148
:10338000012070470020704741780278914201D1B6
:103390000020704740680901401870474178027862
:1033A000914203D0491C0907090F4170704710B5BD
:1033B000002101704170FF2140680131FCF7C7FE18
:1033C00010BD000010B501200349000788600846C1
:1033D000FEF7BAF910BD00009002002010B50349B5
:1033E000002088600846FEF7AFF910BD900200206B
:1033F00070B51E48FFF7C8FF002835D01B4C243C91
:10340000A07A002830D11A491848FFF7CDFB204692
:103410001C300022026002718721017014498B7AEE
:10342000002B01D083230370CB7A002B03D00378C9
:10343000FD252B4003700B7B002B03D003785B082A
:103440005B0003700B78437009798170C270027160
:103450000648FFF7A3FF0549054805220839EC385F
:10346000FEF755FA0120A07270BD00006C0000202C
:103470007C03002010B510210648FCF768FE0121EE
:103480000448022241708270017142710272C1715E
:1034900010BD0000A103002070B50F4DA988A868D9
:1034A000FCF770FF0446E988E868FCF76BFF012829
:1034B00002D0002809D00AE0012C02D0002C02D052
:1034C00005E0032070BD022070BD012C01D000205A
:1034D00070BD012070BD00000400002010B5054C37
:1034E000A060A180E260E38000F0BCF900F0CAF9BE
:1034F00010BD00000400002010B50C4A5378002BCA
:1035000008D01278012A07D0022A08D0032A09D04D
:10351000072010BD012010BD00F00AF810BD00F01A
:103520001DF810BD00F0E2F810BD000004000020FE
:1035300010B5532805D9572803D0582801D00320A7
:1035400010BD002907D01422002100F017FA00282E
:10355000F6D0082010BD80210843F4E710B55928A3
:1035600010D2614A145CFF2C7ED0002902D01422B4
:103570000021ABE014220021F02000F0FFF9002828
:1035800073D1F4E7632816D077285AD00246603A00
:103590001F2A6BD8544A5932101860380478FF2C0F
:1035A00062D000297ED014220021E02000F0E6F94C
:1035B00000285AD188E000291CD014220021E020E4
:1035C00000F0DCF9002850D114220021122000F074
:1035D000D5F9002849D114220021E02000F0CEF9CD
:1035E00000287DD1142200217C2000F0C7F900289A
:1035F00076D110BD14220021E02000F0BFF9002890
:103600006ED114220021F02000F0B8F9002867D113
:10361000142200217C2000F0B1F9002860D114228E
:103620000021E02000F0AAF9002859D1142200213D
:10363000F02000F0A3F9002852D11422002112201A
:10364000D3E70029A6D014220021E12000F096F94A
:10365000002845D114220021104600F08FF90028DF
:103660003ED11422002102E02CE039E03AE077203C
:1036700000F084F9002833D114220021E12000F069
:103680007DF900282CD114220021F02000F076F9D9
:10369000002825D114220021104600F06FF90028DF
:1036A0001ED100E014E014220021F02000F066F9A1
:1036B000002815D114220021772000F05FF900289E
:1036C0000ED110BD022010BD1422012120468CE72E
:1036D00014220021E02000F051F9002800D149E730
:1036E000082010BD032010BDBD45000810B5C3283B
:1036F00001D3052010BD1A4A145CFF2C03D08E2C78
:1037000003D3062010BD022010BD16480129025D1A
:1037100004D0002910D002291BD01EE0022A03D0B9
:10372000012A01D0032A18D114220021204600F0DA
:1037300025F900280BD110E0022A01D0012A0CD172
:1037400014220021F02000F019F90028ECD0082004
:1037500010BD012AE8D0042AE6D0002010BD0000E8
:103760006C44000890000020F3B581B00F4600259E
:103770000126FCF717FE3A4C206107E0FCF712FE29
:103780002169401AB84201D30420FEBDFFF784FE30
:103790000128F3D11220FFF72EF90022A188A0689A
:1037A000FCF7F9FD2420FFF726F90122A188A06883
:1037B000FCF7F1FD1220FFF71EF9E188E068FCF745
:1037C000E1FD012800D135437004060C1220FFF7FB
:1037D00012F90022A188A068FCF7DDFD2420FFF784
:1037E0000AF90122A188A068FCF7D5FD1220FFF795
:1037F00002F9FF2EE1D91220FFF7FDF80022A1887F
:10380000A068FCF7C8FD2420FFF7F5F80122A18885
:10381000A068FCF7C0FD1220FFF7EDF81220FFF7BB
:10382000EAF80022E188E068FCF7B5FD0022A188F3
:10383000A068FCF7B0FD2420FFF7DDF80122A18885
:10384000A068FCF7A8FD1220FFF7D5F80122E18857
:10385000E068FCF7A0FD019805700020FEBD0000A7
:103860000400002010B5064C0122A188A068FCF7D6
:1038700092FD0122E188E068FCF78DFD10BD00009B
:103880000400002010B5054802210170012141709B
:103890008E2203490348FCF741FC10BD04000020C0
:1038A0002F4500089000002038B5FFF7F5FD304C9B
:1038B0000228A07106D00925ED06012806D00328AC
:1038C00037D04EE0FFF7CEFF002038BD0122114671
:1038D0002846FCF760FDFF216846017024480A2154
:1038E000401CFFF741FF69466078FFF777FA6846AA
:1038F0000478FF2C35D020211E48FCF728FC1D48F9
:10390000CD210170014620314978417081218170BB
:10391000E2070121002A00D0C170A20700D5017181
:10392000620700D54171012251031348FCF733FDB2
:1039300017E00F4A0F48121D511E6030FFF727FA9B
:1039400000280ED1012211462846FCF724FD2179DA
:10395000E078FFF7D1FD082805D006486030FFF772
:1039600026FA012038BD0120FCF737FCF9E70000FA
:10397000480000200003002000080048F8B5154664
:103980000E460746144CFCF70DFD206107E0FCF7DE
:1039900009FD2169401AA84201D30420F8BDFFF7B0
:1039A0007BFD0328F3D1FFF759FC206103E0FFF70B
:1039B00073FD0328E7D1FFF751FC2169401A3C2829
:1039C000F5D3002E03D0AF208000FFF714F838465F
:1039D00000F004F8F8BD000004000020F8B5474CE2
:1039E000054601260022E188E068FCF7D4FC12209D
:1039F000FFF701F80022A188A068FCF7CCFC242086
:103A0000FEF7F9FF0122A188A068FCF7C4FC122090
:103A1000FEF7F1FFA188A068FCF7B4FC002868D08D
:103A20000027E80701D0012200E00022E188E068D9
:103A3000FCF7B1FC1220FEF7DEFF0022A188A0688F
:103A4000FCF7A9FC2420FEF7D6FF0122A188A0687C
:103A5000FCF7A1FC1220FEF7CEFFA188A068FCF7BE
:103A600091FC002845D0E807C00F46406D087F1C38
:103A7000082FD6DB002E01D0012200E00022E188D1
:103A8000E068FCF788FC1220FEF7B5FF0022A18851
:103A9000A068FCF780FC2420FEF7ADFF0122A1887E
:103AA000A068FCF778FC1220FEF7A5FFA188A068AB
:103AB000FCF768FC00281CD00122E188E068FCF7D4
:103AC0006AFC1220FEF797FF0022A188A068FCF78D
:103AD00062FC2420FEF78FFF0122A188A068FCF77A
:103AE0005AFC1220FEF787FFC820FEF784FF002053
:103AF000F8BDFFF7B7FE0820F8BD00000400002065
:103B000010B5164C61892069FCF73CFC012805D1F1
:103B10002189E068FCF736FC012806D0618920691C
:103B2000FCF730FC012802D007E0032010BD2189FA
:103B3000E068FCF727FC002806D061892069FCF7C3
:103B400021FC002802D007E0022010BD2189E06896
:103B5000FCF718FC0128F8D0002010BD1800002048
:103B6000F8B5364E054630780C46002804D0B079BA
:103B7000002803D00620F8BD0120F8BD0821601CF4
:103B8000FCF7E5FA0320207008206070A87A00286E
:103B900001D009206070287B0221002802D06078C3
:103BA00008436070E87A0422002802D0607810434D
:103BB000607028681023002802DA6078184360706B
:103BC00068682027002802DA607838436070287817
:103BD000A0702879E0707079032806D0042806D0F8
:103BE000002800D022700020F8BD287A1EE0687BF3
:103BF000002802D0207918432071A87B002802D029
:103C000020793843207109202856002801DD2079C9
:103C100003E0002803DA20790E21084320710820F0
:103C20002856002804DD2079012105E02071D9E71C
:103C30000028D7DA20790F210843F7E71800002081
:103C4000F8B500250E46FF2810D0E63800210127E0
:103C5000584C0300FEF7BEFD11A0A69063619B9B2C
:103C60009B5A9B549B331E1C1A179B0000F03EF975
:103C70001421FA2000F0F5F9FA21AA2000F0E4F965
:103C80001421002075E000F03DF980E021707EE015
:103C900027707CE01421FA2000F0E3F945489621D2
:103CA000401C00F097F800282FD1424920791431A8
:103CB00062780A5407286AD2401C207167E01421F8
:103CC000FA2000F0CEF92179022916D939481430AA
:103CD00040182038C17F50290FD1817F642902D03C
:103CE000C82905D009E0407FC82806D1032003E099
:103CF000407FC82801D1042060711421607938E028
:103D00001421FA2000F0ADF9A771F8BD1421FA20B2
:103D100000F0A7F90220A071F8BDA17137E01421CD
:103D2000FA2000F09EF9A079012800D140252078E2
:103D3000002801D020200543E078022801D110207E
:103D40000543B07A002801D004200543F07A00280A
:103D500001D002200543307B002800D03D431421D0
:103D6000284600F071F91421A07800F06DF91421B3
:103D7000607800F069F9F8BD1421FA2000F071F9BB
:103D80000C489621801C00F025F80028F3D114215E
:103D9000FA2000F066F9F8BD1421FA2000F061F96C
:103DA000E770F8BD1421FA2000F05BF90220E07002
:103DB000F8BD00001800002010B5054CE06021811E
:103DC0002261638100F092F800F080F810BD0000DD
:103DD00018000020F3B581B00F4600250126FCF73E
:103DE000E1FA044606E0FCF7DDFA001BB84201D315
:103DF0000420FEBDFFF784FE0128F4D11220FEF757
:103E0000FAFD314C00222189E068FCF7C4FA242035
:103E1000FEF7F1FD01222189E068FCF7BCFA1220CF
:103E2000FEF7E9FD61892069FCF7ACFA012800D1B1
:103E300035437004060C1220FEF7DDFD00222189B7
:103E4000E068FCF7A8FA2420FEF7D5FD01222189BD
:103E5000E068FCF7A0FA1220FEF7CDFDFF2EE1D9B5
:103E60001220FEF7C8FD00222189E068FCF793FAD2
:103E70002420FEF7C0FD01222189E068FCF78BFABF
:103E80001220FEF7B8FD1220FEF7B5FD0022618971
:103E90002069FCF780FA00222189E068FCF77BFAB0
:103EA0002420FEF7A8FD01222189E068FCF773FABF
:103EB0001220FEF7A0FD012261892069FCF76BFA50
:103EC000019805700020FEBD1800002010B5064CBA
:103ED00001222189E068FCF75EFA012261892069EC
:103EE000FCF759FA10BD00001800002000B500F0E2
:103EF00009F803490020087148618861487100BDD4
:103F000018000020054864214170022181700121C0
:103F1000C1700021017081717047000018000020FD
:103F200070B50546002407E028194078C82100F044
:103F30008BF8002804D1641C2878A042F4DC00200F
:103F400070BD000070B5FFF7DBFD2C4C02286071DE
:103F50002CD00925ED0601282BD0FFF77FF9A169A8
:103F6000401A2749884223D920462430FFF70CFA0B
:103F700000281DD0204623492430FEF715FE214994
:103F800020481C31FFF7ECFD002811D10122114619
:103F90002E462846FCF7FFF91A481C30FFF7C0FFF1
:103FA000002822D0FCF7FEF905461AE0FFF78EFF45
:103FB00070BD012211462846FCF7EDF90F480A2191
:103FC000801CFFF707FF0F49A0781039FFF738FE74
:103FD0000022012128460EE0FCF7E4F9401B1428DA
:103FE00003D8FFF78DFD0328F6D1FFF737F9A0615D
:103FF000002201213046FCF7CEF970BD48000020B8
:10400000881300007C03002070B50546FCF7CAF950
:10401000044606E0FCF7C6F9001BA84201D30420C1
:1040200070BDFFF76DFD0328F4D1FFF717F90446C3
:1040300003E0FFF765FD0328E8D1FFF70FF9001B48
:104040003C28F6D3002070BD10B504460846FFF7A3
:10405000DBFF002801D0042010BD204600F012F83C
:1040600010BD10B504460846FFF7CEFF002801D06A
:10407000042010BDAF208000FEF7BDFC204600F0FC
:1040800001F810BDF8B5474C0546012600226189AC
:104090002069FCF780F91220FEF7ADFC002221898F
:1040A000E068FCF778F92420FEF7A5FC01222189BD
:1040B000E068FCF770F91220FEF79DFC2189E068AA
:1040C000FCF760F9002868D00027E80701D001223A
:1040D00000E0002261892069FCF75DF91220FEF7FB
:1040E0008AFC00222189E068FCF755F92420FEF7BC
:1040F00082FC01222189E068FCF74DF91220FEF7CD
:104100007AFC2189E068FCF73DF9002845D0E807F2
:10411000C00F46406D087F1C082FD6DB002E01D053
:10412000012200E0002261892069FCF734F91220A5
:10413000FEF761FC00222189E068FCF72CF92420BD
:10414000FEF759FC01222189E068FCF724F91220CE
:10415000FEF751FC2189E068FCF714F900281CD017
:10416000012261892069FCF716F91220FEF743FC51
:1041700000222189E068FCF70EF92420FEF73BFCC1
:1041800001222189E068FCF706F91220FEF733FCD2
:10419000FA20FEF730FC0020F8BDFFF797FE08205C
:1041A000F8BD00001800002011A0FEF703FB134D1E
:1041B0000024295D12A0FEF7FDFA641C202CF8DB18
:1041C00010A0FEF7F7FA134D002408212846FCF74B
:1041D000DEF86420FCF701F8641C642CF5DBBFF307
:1041E0004F8F0E490C48C860BFF34F8F00BFFDE7EB
:1041F000535049204552524F520A000020030020DC
:10420000256420000A7265626F6F74696E672E2ED6
:104210002E0A0000000400480400FA0500ED00E04A
:1042200070B50646FCF7BEF80446084D06E0FCF7FC
:10423000B9F8001BB04201D9042070BD2988686814
:10424000FCF7A0F80028F2D0002070BD3400002058
:1042500010B50E4C21886068FCF794F8012802D153
:10426000FCF7A0F8E060FCF79DF8E168401A14281C
:104270000BD9C820FFF7D4FF1420FBF7AEFFAA200C
:1042800000F094F80A20FBF7A8FF10BD34000020CE
:1042900010B500F05DF8FCF785F80149C86010BD65
:1042A0003400002010B5034C60602180A260638060
:1042B00010BD00003400002070B5044666380300CD
:1042C000FEF788FA0A1406080A0C0E101216181ABD
:1042D000482413E0492411E04B240FE04D240DE065
:1042E0004F240BE0502409E0512407E0472405E067
:1042F000522403E0532401E0532C0BD8022902D0AE
:1043000000290DD00EE0FCF74DF8084D2969401A40
:10431000502801D8002070BDFCF744F8286101E066
:1043200080200443204600F041F870BD3400002096
:1043300010B5064C012221886068FCF72CF8012298
:104340006188A068FCF727F810BD00003400002049
:1043500010B5064C012221886068FCF71CF8002289
:104360006188A068FCF717F810BD00003400002039
:1043700010B5FFF76DFF0B4A0B48511EFEF707FD06
:1043800000280AD10748001F0179C078FFF794FF81
:10439000452803D00448FEF70AFD10BD0120FBF7B5
:1043A0001CFF10BD4C0000206003002070B52E4C97
:1043B000054621886068FBF7E5FF00282AD0002227
:1043C00021886068FBF7E7FF0520FEF714FB012258
:1043D0006188A068FBF7DFFF6E20FEF70CFB6188A9
:1043E000A068FBF7CFFF002814D001222188606865
:1043F000FBF7D1FF4120FEF7FEFA0022218860681A
:10440000FBF7C9FF1E20FEF7F6FA0026E80705D0E5
:10441000012204E0FFF79CFF452070BD0022618867
:10442000A068FBF7B8FF012221886068FBF7B3FFA3
:104430004120FEF7E0FA002221886068FBF7ABFF1D
:104440001E20FEF7D8FA6D08761C082EDEDB01224E
:1044500021886068FBF79FFF00226188A068FBF756
:104460009AFF002070BD000034000020FF08161ED7
:1044700026252E363D3E46454E55660D151D242DEE
:104480002C353C43444D545B5A111C1B232B3433B5
:104490003B424B4C520E125C1A22212A32313A41D5
:1044A000494A597E192914070F171F272F373F47ED
:1044B0004F765F6C757D4E6B73747C69727A707128
:1044C000FFFF13565EFFFFFFFFFFFFFF79584A57BC
:1044D00039FF6E636F616A65606D6764FFFFFFFFA0
:1044E000FFFFFF62FFFFFFFFFF8B8C8DFFFFFFFFD2
:1044F000FFFFFFFFFFFFFFFFFFFFFFFFFFFFFFFFCC
:10450000FFFFFFFFFFFFFFFFFFFFFFFFFFFFFFFFBB
:10451000FFFFFFFFFFFFFFFFFFFFFFFFFFFFFFFFAB
:10452000FFFFFF08101820283038404850575F011F
:104530000101010101010303010101010101030165
:104540000202010201010301020101010101030153
:104550000101010101010301010101010101030147
:104560000101010101010301030101010101030135
:104570000101010101010301010101010101030127
:104580000101010101030303020101010103030110
:1045900001030101030103010301030303030303F7
:1045A00003030303030303010303010103030101E5
:1045B00001010103010101010101010101FF761661
:1045C0001E26252E363D3E46454E55660D151D24AC
:1045D0002D2C353C43444D545B5A141C1B232B3467
:1045E000333B424B4C520E125D1A22212A32313A91
:1045F00041494A597C1129580506040C030B830ACA
:104600000109777E6C757D7B6B73747969727A7042
:1046100071FFFF6178075A144AFF11FF6C757D6BBB
:104620007469727A7071FFFFFFFFFFFFFFFFFFFFEA
:10463000FFFFFF1F272F0001060755534234564343
:104640002050726F746F636F6C20426F6172640AE6
:1046500049424D20504320436F6D70617469626C14
:10466000650A64656B754E756B656D20323032324C
:10467000000000000000000000010203040607081B
:10468000090000000001020304000000AC4600081D
:104690000000002090000000EE2700083C470008C2
:1046A0009000002028090000FE27000800000000FC
:1046B00002010000000000000000000000000000F7
:1046C00000000000000000000000000000000000EA
:1046D00000000000000000000000000000000000DA
:1046E00000000000000000000000000000000000CA
:1046F00000000000000000000000000000000000BA
:1047000000000000000000000000000000000000A9
:104710000000000000000000000000000000000099
:1047200000000000000000000000000000127A00FD
:0C4730000000000000000000000000007D
:04000005080000C12E
:00000001FF
